S0120000626F6F746C6F616465722E73726563E7
S21401F0000C9446F80C9463F80C9463F80C9463F82B
S21401F0100C9463F80C9463F80C9463F80C9463F8FE
S21401F0200C9463F80C9463F80C9463F80C9463F8EE
S21401F0300C9463F80C9463F80C9463F80C9463F8DE
S21401F0400C9463F80C9463F80C9463F80C9463F8CE
S21401F0500C9463F80C9463F80C9463F80C9463F8BE
S21401F0600C9463F80C9463F80C9463F80C9463F8AE
S21401F0700C9463F80C9463F80C9463F80C9463F89E
S21401F0800C9463F80C9463F80C9463F811241FBE77
S21401F090CFEFD0E1DEBFCDBF11E0A0E0B1E0E8E305
S21401F0A0FCEF01E00BBF02C007900D92A030B10744
S21401F0B0D9F711E0A0E0B1E001C01D92A030B10780
S21401F0C0E1F70C941FFD0C9400F800000000089571
S21401F0D085B7806285BF889508951ABA17BA11BA9E
S21401F0E082E082B983B9D29AD09AD19A8B989FE757
S21401F0F08091610089238093610082B1892382B95E
S21401F100A79AA69AA59AA49AA39AA29AA19AA09A0D
S21401F1108D9A8F9A8E9ABB9887B3892387BB159A47
S21401F120D79AD39A1D9ADF9ADA9A0895992780FF7B
S21401F13002C0DA9801C0DA9A81FF02C0D99801C0EC
S21401F140D99A82FF02C0D8980895D89A08951F9335
S21401F150CF93C7E010E08C2F0E9496F827E030E0AE
S21401F1608FEF9FE70197F1F72150304037FFF8CF37
S21401F170C6951F5F133078F38C2F0E9496F8CF91B7
S21401F1801F910895CF93C0E087E00E9496F823E090
S21401F19030E08FEF9FE70197F1F72150304037FFBE
S21401F1A0F8CF80E00E9496F823E030E08FEF9FE7EB
S21401F1B00197F1F72150304037FFF8CFCF5FC330CA
S21401F1C018F3CF91089587FF02C0DF9A01C0DF9838
S21401F1D0880F99270895880FCE99816099270895F9
S21401F1E00F931F93CF93082FC0E01C2F802F0E94F0
S21401F1F0E3F8082FDB9A8C2F0E94EBF8C82FDB98D8
S21401F2001F5F183098F39927CF911F910F9108959A
S21401F210EF92FF921F93CF93DF93CDB7DEB724977C
S21401F2200FB6F894DEBF0FBECDBF9C0140E050E0A4
S21401F23088E68983FE013196C901880F892F881FC8
S21401F240990B91958F708183822F880F8B834C83C6
S21401F250DB981D98142F7F01F70181917F010E9491
S21401F260F0F81F5F1430C0F310E080E00E94F0F861
S21401F2701F5F1430D0F3DB9ADB9824960FB6F89410
S21401F280DEBF0FBECDBFDF91CF911F91FF90EF90F4
S21401F29008951D9A0895EF92FF920F931F93CF93AF
S21401F2A0DF93EC01E880F9800A811B81D801C70150
S21401F2B09070A070B0700097A105B10541F40E944E
S21401F2C049F9BB27A12F902F8F2D0E9408F908948A
S21401F2D0E11CF11C011D111DE882F9820A831B83C2
S21401F2E080E00E94F0F89927DF91CF911F910F914E
S21401F2F0FF90EF90089588E190E029E00FB6F8942A
S21401F300A89581BD0FBE21BDFFCFAF92BF92CF9210
S21401F310DF92EF92FF920F931F93CF93DF935C01DF
S21401F3206A017B01E9014050504F6140704018F07E
S21401F33080E090E023C082EF9FE00E9403FE8C01F4
S21401F34084EF9FE00E9403FE0817190779F08F5F8C
S21401F3509F4F61F06FEF84EF9FE00E9410FE6FEF0A
S21401F36085EF9FE00E9410FEE199FECF9E01B70156
S21401F370A601C5010E946AFD81E090E0DF91CF9170
S21401F3801F910F91FF90EF90DF90CF90BF90AF90BD
S21401F39008952F923F924F925F926F927F928F9233
S21401F3A09F92AF92BF92CF92DF92EF92FF920F930E
S21401F3B01F93CF93DF93CDB7DEB7C450D1400FB6BE
S21401F3C0F894DEBF0FBECDBFDC01CB01BA2FA92F4B
S21401F3D0982F8827FE01EF5FFE4F80839183A283DB
S21401F3E0B383AA24BB246501150126018601750194
S21401F3F0CE018F5F9E4F0E944BF99927AA27BB2704
S21401F4000E2C04C0880F991FAA1FBB1F0A94D2F79F
S21401F410282A392A4A2A5B2A0894A11CB11CC11C35
S21401F420D11C88E090E0A0E0B0E0E80EF91E0A1FCB
S21401F4301B1F94E0A916B104C104D104C8F26624C6
S21401F440772443016401530184017301CE018F5F68
S21401F4509E4F0E944BF99927AA27BB270E2C04C062
S21401F460880F991FAA1FBB1F0A94D2F7682A792A08
S21401F4708A2A9B2A0894A11CB11CC11CD11C88E0B5
S21401F48090E0A0E0B0E0E80EF91E0A1F1B1F94E012
S21401F490A916B104C104D104C8F26114710481042F
S21401F4A0910409F4DCC0AA24BB246501A614B704A0
S21401F4B0C804D90408F04AC0A114B104C104D10497
S21401F4C021F1D201C1019070A070B0700097A10522
S21401F4D0B105D9F41127052DF42CE32C0894E10885
S21401F4E0F108010911098E2D0E9496F8B02FAF2D53
S21401F4F09E2D882720E031E0AC01BD01CE010196AA
S21401F5000E9485F9882309F445C0D201C101907093
S21401F510A070B0708E010F5F1F4F080F191FCE012C
S21401F5208F5F9E4F0E944BF9D8018C930894A11CC3
S21401F530B11CC11CD11C0894211C311C411C511C3E
S21401F540A614B704C804D90408F4B6CF1127052DAC
S21401F550F42CE32C8FEF90E0A0E0B0E028223922D3
S21401F5604A225B22211431044104510429F40894EF
S21401F570E108F10801091109B02FAF2D9E2D88274A
S21401F58020E031E0AC01BD01CE0101960E9485F973
S21401F590882319F480E090E066C0AA24BB246501A4
S21401F5A01501260186017501CE018F5F9E4F0E94CF
S21401F5B04BF99927AA27BB270E2C04C0880F991F41
S21401F5C0AA1FBB1F0A94D2F7282A392A4A2A5B2A7D
S21401F5D00894A11CB11CC11CD11C88E090E0A0E0DD
S21401F5E0B0E0E80EF91E0A1F1B1F94E0A916B1042D
S21401F5F0C104D104C8F2662477244301640153018F
S21401F60084017301CE018F5F9E4F0E944BF99927AB
S21401F610AA27BB270E2C04C0880F991FAA1FBB1F41
S21401F6200A94D2F7682A792A8A2A9B2A0894A11C66
S21401F630B11CC11CD11C88E090E0A0E0B0E0E80E4F
S21401F640F91E0A1F1B1F94E0A916B104C104D104B8
S21401F650C8F2611471048104910409F024CF0E9458
S21401F66049F981E090E0CC5FDE4F0FB6F894DEBF3B
S21401F6700FBECDBFDF91CF911F910F91FF90EF90FD
S21401F680DF90CF90BF90AF909F908F907F906F90BC
S21401F6905F904F903F902F9008950F931F93CF93B5
S21401F6A0DF938C010E9403FEEC0121968E5F9F4F33
S21401F6B070F46C2FC8010E9410FE8D2F99270F5FE2
S21401F6C01F4F682FC8010E9410FEE199FECFDF91FF
S21401F6D0CF911F910F910895FF920F931F93F82ECC
S21401F6E08CEE9FE00E9403FE8C0183E0000F111F49
S21401F6F08A95E1F78F2D992787709070082B192B23
S21401F700602F8CEE9FE00E9410FE812F9927682FB4
S21401F7108DEE9FE00E9410FEE199FECF1F910F91A2
S21401F720FF9008958EEF9FE00E94FBFD8460682F96
S21401F7308EEF9FE00E9410FEE199FECF0895EF92B2
S21401F740FF920F931F9381EF9FE00E94FBFD8F3F77
S21401F75019F0682F6F5F01C061E0162F80EF9FE000
S21401F7600E94FBFD082F153008F459C08F3F61F148
S21401F7706FEF80EF9FE00E9410FEE199FECF84EFCD
S21401F7809FE00E9403FEAA27BB278F5F9F4FA040E2
S21401F790B04091F48EEF9FE00E94FBFD80FD03C018
S21401F7A00E94C2F8FDCF65E081EF9FE00E9410FE47
S21401F7B0E199FECF0E947BF96FEF81EF9FE00E94F7
S21401F7C010FEE199FECF2BC08EEF9FE00E94FBFD5D
S21401F7D080FD25C00E94C2F860E082EF9FE00E9493
S21401F7E010FE60E083EF9FE00E9410FEE199FECFDD
S21401F7F060E070E080E090E00E94C9F9882321F47F
S21401F8000E9492FB0E947BF960E084EF9FE00E94D9
S21401F81010FE60E085EF9FE00E9410FE1FEF612F53
S21401F82081EF9FE00E9410FEE199FECF0F3F59F154
S21401F83082EF9FE00E9403FE7C0100271127C8018A
S21401F840B7010E94C9F9882321F40E9492FB0E9405
S21401F8507BF96E2D84EF9FE00E9410FEBB27A12F3F
S21401F860902F8F2D682F85EF9FE00E9410FE6FEF7F
S21401F87080EF9FE00E9410FE6FEF81EF9FE00E94F5
S21401F88010FEE199FECF0E94A7F86FEF81EF9FE08F
S21401F8900E9410FEE199FECF0C9400001F910F917B
S21401F8A0FF90EF9008958CEE9FE00E9403FE8F5F1D
S21401F8B09F4F09F048C060E080EE9FE00E9410FE76
S21401F8C060E081EE9FE00E9410FE60E084EE9FE023
S21401F8D00E9410FE60E085EE9FE00E9410FE60E050
S21401F8E086EE9FE00E9410FE60E087EE9FE00E9499
S21401F8F010FE60E082EE9FE00E9410FE60E083EE64
S21401F9009FE00E9410FE60E088EE9FE00E9410FEDD
S21401F91060E089EE9FE00E9410FE60E08AEE9FE0C4
S21401F9200E9410FE60E08BEE9FE00E9410FE60E0F9
S21401F9308CEE9FE00E9410FE60E08DEE9FE00E943C
S21401F94010FEE199FECF04B603FE13C08EEF9FE0D2
S21401F9500E94FBFD81FD0DC08EEF9FE00E94FBFD26
S21401F96082FD07C080EE9FE00E944DFB81E00E9471
S21401F9706CFB04B600FE07C084EE9FE00E944DFBC0
S21401F98083E00E946CFB04B602FE07C086EE9FE091
S21401F9900E944DFB84E00E946CFB04B601FE10C081
S21401F9A004B600FC0DC08EEF9FE00E94FBFD81FDBA
S21401F9B007C082EE9FE00E944DFB82E00E946CFB36
S21401F9C08EEF9FE00E94FBFD81FF07C08AEE9FE05D
S21401F9D00E944DFB86E00E946CFB8EEF9FE00E942A
S21401F9E0FBFD82FF07C088EE9FE00E944DFB85E08D
S21401F9F00E946CFB84B7877F84BF84B78E7F84BFE9
S21401FA0084B78B7F84BF84B78D7F84BF8EEF9FE0E2
S21401FA100E94FBFD8D7F682F8EEF9FE00E9410FEF7
S21401FA20E199FECF8EEF9FE00E94FBFD8B7F682F52
S21401FA308EEF9FE00E9410FEE199FECF0895CFEF72
S21401FA40D0E1DEBFCDBFF89488E190E020E00FB6AC
S21401FA50F894A89581BD0FBE21BD0E946DF80E9445
S21401FA6053FC85E899EF2C0166247724AA24BB244D
S21401FA70C6EFDFE0450173016201082C04C0F6946D
S21401FA80E794D794C7940A94D2F7CE010E94FBFD5F
S21401FA90C81621F06C2DCE010E9410FE0894A11C00
S21401FAA0B11C88E090E0880E991E219694E0A91674
S21401FAB0B10408F30E949FFB80E090E00C941BFECB
S21401FAC084B195B1089500000895009711F001974B
S21401FAD0F1F708958F929F92AF92BF92CF92DF92E5
S21401FAE0EF92FF920F931F93CF93DF934C017A010E
S21401FAF08B018091680080FDFCCFE199FECF83E009
S21401FB00F70100935B0080936800E8958091680098
S21401FB1086FF0EC08091680080FDFCCFE199FECF84
S21401FB2081E180936800E8958091680086FDF2CFB8
S21401FB30AA24BB246501E901D695C795CE01AA275B
S21401FB40BB27A816B906CA06DB0648F5B801A70101
S21401FB508091680080FDFCCFE199FECF21E0F501A0
S21401FB60EA0DFB1DE80DF91D808191810C01FA015A
S21401FB7060935B0020936800E89511240894A11C0B
S21401FB80B11CC11CD11C4E5F5F4F6F4F7F4FCE0122
S21401FB90AA27BB27A816B906CA06DB06C8F28091B3
S21401FBA0680080FDFCCFE199FECF85E0F701009368
S21401FBB05B0080936800E8958091680086FF0EC020
S21401FBC08091680080FDFCCFE199FECF81E18093B2
S21401FBD06800E8958091680086FDF2CFDF91CF91AD
S21401FBE01F910F91FF90EF90DF90CF90BF90AF9055
S21401FBF09F908F900895E199FECF9FBB8EBBE09AB0
S21401FC0099278DB30895E199FECF9FBB8EBBE09AED
S21401FC1001960DB29FBB8EBBE09A802D9DB30895D1
S21401FC20E199FECF9FBB8EBB6DBB0FB6F894E29AEF
S20C01FC30E19A0FBE0895FFCF13
S80401F0000A
